:10000000B20154290408A700061086108610831632
:10001000061086108610870183122708B2182B2835
:100020003A30A100983017213330A6003E2013301B
:10003000A100883017213E20643016213E20643014
:10004000162138302A200C302A2006302A20B214FB
:1000500027082B283214A600321C39288610033CAE
:10006000031C3E283E200730A100D0301721031486
:1000700008003214FE3C03194F2986140614260882
:1000800087000000321006103230162103140800D9
:10009000003803194F29A80020088400211883176D
:1000A000A001A101A81B5C280008A000A81C4F29E2
:1000B000840A0008A1004F29F4200005031DA00AAE
:1000C0004F296400772003186128B620A801083062
:1000D000A300B72077200318A80AAB1EA801A20C22
:1000E000A30B6928AB1AA213B72022080800360810
:1000F0008400340884178004841300052B1B340605
:10010000FF3E0800A401A501B3124A21D33E031902
:10011000B3162D3EC63E031885280A3E031C8528CB
:10012000A2000310240DA000250DA100200DA10D9B
:10013000A4070318A10A2108A507A40DA50D2208EC
:10014000A4070318A50AA9030319AD284A21C63E2E
:100150000318AD280A3E03189028B31EB428A4093A
:10016000A509A40A0319A50A24084F2933172B0847
:100170001F39003EA1002A080E3E0318A10A331FB2
:1001800017293313A000023029211729B313290896
:100190000319B3170530A8002730A3001030DC2066
:1001A0000330A300E830DC20A3016430DC20A3018D
:1001B0000A30DC202408E328A2002508A100240836
:1001C000A0002E212008A000A8030319B3132908BA
:1001D0000319ED282802031808002008031DB31393
:1001E000B31B0800303E4A2901308A00280807392D
:0201F0000029E4
:10020000820701340234043408341034203440347A
:100210008034A301A200FF30A207031CA307031C24
:100220004F290330A100E63017210B29A101FC3E24
:10023000A000A109031C2229FF300000A007031819
:100240001D29A0076400A10F1C2908000310A10CA0
:10025000A00CFF3E0318262920084F29A501A40160
:100260001030A600210DA40DA50D2208A40223081C
:10027000031C230FA502031844292208A4072308FE
:100280000318230FA5070310A00DA10DA60B3229FB
:1002900020084F29840031088A0030088200831327
:1002A0000313831264000800831607309F00831233
:1002B000C401051483160510831285148316851056
:1002C0008312851583168511831206118316061174
:1002D000051485148515061583128512831685125B
:1002E00083120130A300F4300A218516831685128B
:1002F00083120130A300F4300A216400051882291A
:10030000441083294414640085188829C41089295D
:10031000C414640085198E2944118F294415640082
:1003200004304402031C99290430C4024E30C60034
:100330009B295430C6004408A200033C031CC0297A
:100340000310220DA207B021A000A20AB021A10033
:10035000A20AB02148202008C0002108C100C029FD
:1003600001308A00220882072034003400342D3402
:10037000033400348C3401340034543400340034F9
:100380004408A200033C031CE5290310220DA20728
:10039000D521A000A20AD521A100A20AD52148207A
:1003A0002008C2002108C300E52901308A00220884
:1003B000820700344B340034B034043400346034E9
:1003C00009340034803425340034640046084E3C3F
:1003D000031DEB29411784232030CA000630B600E4
:1003E0000430B4004008AA004108AB0061200D3C75
:1003F000031DF6296120CC000630B6000430B4009D
:100400004008AA004108AB006120CA0064004A0805
:100410005C3C031D0C2A422A64004A085D3C031D13
:10042000122A8A2A64004A085B3C031D182A9C2A67
:1004300064004A08083C031D282AFE3003201030BF
:10044000032020300320FE30032010300320412AF7
:1004500064004A08093C031D392A0130C9006400C0
:10046000063049020318382A20300320C90F2F2AEA
:10047000412A64004A080D3C031D3F2A412A4A08CC
:100480000320FC290630B6000430B4004008AA005E
:100490004108AB000330A9006130B000B1018220F7
:1004A000CB0064004B08013C031D5D2AFE30032095
:1004B000013003201E300921892A64004B08803C4A
:1004C000031D672AFE30032080300320892A640040
:1004D0004B08C03C031D712AFE300320C0300320AE
:1004E000892A64004B08943C031D7B2AFE300320BC
:1004F00094300320892A64004B08D43C031D852ACC
:10050000FE300320D4300320892AFE3003204B081C
:100510000320FC290630B6000430B4004008AA00CD
:100520004108AB000330A9006130B000B101822066
:10053000CB004B080320FC290630B6000430B40081
:100540004008AA004108AB000230A9006130B000A9
:10055000B1018220CB0064004B081E3C031DB52A6C
:1005600086118316861183127A2B64004B081F3C78
:10057000031DBF2A86158316861183127A2B640009
:100580004B08283C031DC92A061283160612831243
:100590007A2B64004B08293C031DD32A06168316C8
:1005A000061283127A2B64004B08323C031DDD2AAD
:1005B00086128316861283127A2B64004B08333C12
:1005C000031DE72A86168316861283127A2B64008F
:1005D0004B083C3C031DF12A0613831606138312B5
:1005E0007A2B64004B083D3C031DFB2A061783163B
:1005F000061383127A2B64004B08463C031D052B1F
:1006000086138316861383127A2B64004B08473CAB
:10061000031D0F2B86178316861383127A2B640013
:100620004B08623C031D742B0630B6000430B40046
:100630004008AA004108AB000330A9006130B000B7
:10064000B1018220C5000230A9006130B000B101C3
:100650008220B8000230A9006130B000B1018220D0
:10066000B9000230A9006130B000B1018220BA00A7
:100670000230A9006130B000B1018220BB0002301D
:10068000A9006130B000B1018220BC000230A90095
:100690006130B000B1018220BD000230A90061309C
:1006A000B000B1018220BE000230A9006130B0006C
:1006B000B1018220BF00FE30032045080320380826
:1006C0000320390803203A0803203B0803203C0894
:1006D00003203D0803203E0803203F080320FE308E
:1006E0000320803003207A2B64004B08633C031DF9
:1006F0007A2B4D24FC2963007B2BFE300320013034
:1007000003201E30092108008516831685128701F3
:1007100083120130A3002C300A21FE300320403028
:1007200003200030032004300320023003201F3058
:100730000320023003200430032000300320003067
:100740000320FE30032080300320FE300320483099
:1007500003200030032004300320083003201F3022
:100760000320083003200430032000300320003031
:100770000320FE30032080300320FE300320503061
:10078000032000300320043003200E3003201530F6
:100790000320043003200430032000300320003005
:1007A0000320FE30032080300320FE300320583029
:1007B00003200030032000300320043003200430E5
:1007C0000320153003200E300320043003200030B6
:1007D0000320FE30032080300320FE3003206030F1
:1007E00003201F300320113003201130032011306B
:1007F00003201130032011300320113003201F305B
:100800000320FE30032080300320FE3003206830B8
:100810000320043003200E3003201F30032000305B
:100820000320003003201F3003200E30032004304B
:100830000320FE30032080300320FE300320703080
:10084000032002300320063003200E3003201E3028
:1008500003200E3003200630032002300320003036
:100860000320FE30032080300320FE300320783048
:100870000320083003200C3003200E3003200F30FB
:1008800003200E3003200C300320083003200030FA
:100890000320FE30032080300320FE30032001308F
:1008A000032032300921FE300320803003205330F2
:1008B000032065300320723003206930032061304B
:1008C00003206C30032020300320433003204C30C1
:1008D00003204330032044300320203003207630AF
:1008E0000320313003202E30032030300320FE302F
:1008F0000320C030032042300320613003207530D4
:100900000320643003203A300320203003204608BF
:100910000320A9014208A4004308A5000230B0004A
:0E092000B101C620FE30032002300320080083
:02400E00753FFC
:00000001FF
